:020000020000FC
:100000000C942B000C942A000C942A000C942A00C7
:100010000C942A000C942A000C942A000C942A00B8
:100020000C942A000C942A000C942A000C942A00A8
:100030000C942A000C942A000C942A000C942A0098
:100040000C942A000C942A000C942A000C942A0088
:100050000C942A0018956FE578E06DBF7EBF789408
:1000600060E0862E63E0962E6CE0A62E6FE0B62E42
:1000700060E3C62E63E3D62E6CE3E62E6FE3F62E26
:1000800060E4562E60E8662E60EC762E6FEF64BB5F
:1000900085BA0E9457000000000000000000000028
:1000A000000000000000000000000C9449007CE00B
:1000B0000E94AE0063E00E94B40100007A95C1F78F
:1000C00079E10E94B80063E00E94B40100007A95D3
:1000D000C1F770E50E94C20063E00E94B401000015
:1000E0007A95C1F778E20E94C20064E00E94B401F0
:1000F00000000E94B80063E00E94B40100007A95FD
:1001000091F770E50E94B80063E00E94B40100001E
:100110007A95C1F778E20E94920164E00E94B401EE
:1001200000000E94B80063E00E94B40100007A95CC
:1001300091F770E50E94920163E00E94B401000013
:100140007A95C1F77CE00E94B80063E00E94B40198
:1001500000007A95C1F70E94B800089575BA67E06B
:100160000E94B40165BA61EB0E94B40165BA0895BA
:1001700055BA67E00E94B40185BA61EB0E94B401F0
:1001800085BA089555BA67E00E94B40185BA61E165
:100190000E94B401F5BA85BAF5BA000085BA00002C
:1001A000F5BA00000000000085BA00000000000061
:1001B000F5BA000000000000000000000000000090
:1001C00085BA0000000000000000000000000000F0
:1001D000F5BA62E00E94B401000085BA62E00E94B4
:1001E000B4010000F5BA67E00E94B401000000000D
:1001F00085BA67E00E94B40100000000C5BAE5BA04
:10020000A5BAB5BA95BAD5BA85BAC5BA0000E5BAE5
:100210000000A5BA0000B5BA000095BA0000D5BA32
:10022000000085BA0000C5BA000000000000E5BA71
:10023000000000000000A5BA000000000000B5BAF0
:1002400000000000000095BA000000000000D5BAD0
:1002500000000000000085BA000000000000C5BAE0
:100260000000000000000000000000000000E5BAEF
:100270000000000000000000000000000000A5BA1F
:100280000000000000000000000000000000B5BAFF
:10029000000000000000000000000000000095BA0F
:1002A0000000000000000000000000000000D5BABF
:1002B000000000000000000000000000000085BAFF
:1002C0000000000000000000000000000000F5BA7F
:1002D00085BAF5BA85BAF5BA85BAF5BA85BAF5BA66
:1002E00085BA67E00E94B40195BA67E00E94B40144
:1002F000A5BA67E00E94B401B5BA67E00E94B401F4
:10030000C5BA67E00E94B401D5BA67E00E94B401A3
:10031000E5BA67E00E94B401F5BA67E00E94B40153
:1003200085BA089555BA67E00E94B40185BA61E1C3
:100330000E94B401F5BA00006FE085BA00006A952A
:10034000F5BAD9F7000085BA80E06FE385BB8395E5
:1003500000006A95D9F7000085BB0000000000008E
:0E0360000000000085BA08956A95F1F708952F
:00000001FF
